:100000006F20400B00000000B81D0000BA1D00006A
:1000100000000000000000000000000000000000E0
:1000200000000000000000000000000000000000D0
:10003000BC1D000000000000842000000000000043
:1000400086200000882000008A2000008C2000000C
:100050008E200000902000009220000094200000DC
:1000600096200000982000009A2000009C200000AC
:100070009E200000A0200000A2200000A42000007C
:10008000A6200000A8200000AA200000AC2000004C
:10009000AE200000B0200000B220000000000000F0
:1000A000511126C022C206C4828282441244A24058
:1000B000310182802A86014593F6150091C232955E
:1000C00085810606F5F9828000000000634E050276
:1000D00063C305042E86AA857D5515C285466378BF
:1000E000B6006356C00006068606E36CB6FE014500
:1000F00063E4C500918D558D85820582F5FA828075
:100100008682C93F2E8582823305A04063D70500D1
:10011000B305B040C1B7B305B0408682653F330533
:10012000A0408282868263C70500634905005D376F
:100130002E858282B305B040E35B05FE3305A04007
:10014000513F3305B040828200003D432A876373EC
:10015000C3029377F700BDEFADE5937606FF3D8AC6
:10016000BA960CC34CC30CC74CC74107E36BD7FE10
:1001700011E28280B306C3408A0697020000969679
:100180006780A6002307B700A306B7002306B700C1
:10019000A305B7002305B700A304B7002304B700E5
:1001A000A303B7002303B700A302B7002302B700DD
:1001B000A301B7002301B700A300B7002300B700D5
:1001C000828093F5F50F93968500D58D9396050162
:1001D000D58D61B793962700970200009696868288
:1001E000E78086FA9680C1171D8F3E96E374C3F8A8
:1001F000A5B7EFF2FFEA2E869305100AEF00F00E86
:100200006DB5EFF2FFE9711137170140A1462EC01D
:1002100014CBB2849305000A1306E00A2A84EF0087
:10022000D00C824722859305000A3E86EF00F00B32
:10023000A68522857D3F11018DBD19CEEFF25FE6C7
:10024000C1479376F60F63F3C700C1462E86930528
:100250000009EF00207091BD8280EFF27FE491E110
:1002600085459205C51593F5F50FEF00A06E35BDD8
:10027000EFF21FE31301C1FD614681456800F135CE
:10028000116502C002C202C4EF20C0383715014018
:10029000A1478A8513050540372401407C8002C4AC
:1002A000EF20A00E13050440EF101069B7070E00F1
:1002B0003ECC6C008547130504402300F10202C6C2
:1002C00002C802CA02CEEF1090699D4605469145CC
:1002D00013050440EF1050729946054681451305F9
:1002E0000440EF10B07EB705000213050440EF2074
:1002F000E007854513050440EF10506B13050440DB
:10030000EF10D06B930404402685EF10D06B6DFD89
:100310001305044037240140EF10706B13040440B0
:100320002285EF10706B6DFD13014102BDBB3707D5
:100330000020130747059306070281471223090788
:10034000B297C207C183E31BD7FE91833707002012
:100350002318F7048280EFF2BFD43725014085458A
:1003600013050540EF10D06789B3EFF27FD3B727AD
:100370000140894513850740EF10B07E2DC11384DD
:1003800041820620B72701401385074013871400D8
:100390001AA0EF101072B707002086049387470554
:1003A000A6978AA31E20BD8B1EA091E34937372450
:1003B0000140832744401304044093F7074085C35A
:1003C00091452285EF10F07919C9D1452285EF10AA
:1003D00090772393A18281452285EF10106EF1B1B1
:1003E000EFF21FCCB707002083D707051307700271
:1003F000138587FD6363F70001459305803D2A055A
:10040000D13909811345F5FF1375F50F79B90567E2
:1004100093878182130747509AA313074040DAABB2
:100420003717014018471377070219E3314798A39C
:100430008280EFF2FFC6138481828144B7170140A6
:1004400088471C308546182093F50701BD8BB3976C
:10045000F600E98F93F7F70F13768700C9E3C9C158
:100460003E20C165FD156384B70085073EA03E2090
:10047000954563FEF5049375170085E193671600B3
:100480001CA01C44A9C721E6268582971C2093E75F
:1004900007011CA02DA8854455B74E2063E9B7027B
:1004A0009377270099C37E209DC35C441367270080
:1004B00018A081CB19E6268582971C2093E70702B6
:1004C0001CA07A203E2063F9E70023110400854731
:1004D0005104E392F4FCD1BE998F3EA0CDBFC9D1A7
:1004E000118B75F791471CA01C4823110400E5D31C
:1004F00079FE268582971C2093E7070459BF814720
:10050000014513870185B9463306F7001022850798
:10051000329542054181E399D7FE8280EFF25FB8C0
:1005200013860185AA84D1468145014541209387E0
:100530000185984BB7E72420938727C3138401854F
:100540006317F7006D3F7E246393A7009DC4930754
:1005500000401EA0B72708C0938727905CC0B7074C
:1005600005F49387F7671CC4A3010400493FB7E76C
:100570002420938727C36AA41CC805BEEFF25FB28C
:10058000BD3F13840185B7E72420938727C36AA45E
:10059000C14613860185814501451CC80520C14619
:1005A00013060401C1450145112801B6EFF25FAF02
:1005B000060539891365050A4D22C5BCEFF25FAE09
:1005C000B7E700E005671314150023A0E718398882
:1005D000B71701401307000451111364040AD8CB64
:1005E000228536C432C22EC0212B82451246A24635
:1005F00065D9228585262285212375DDB71701401F
:100600001307000498CBB7F700E023A4070023A248
:1006100007000567B7E700E023A0E710310171B4D8
:10062000EFF21FA83111B68491E590A310A390A218
:100630005101A5BC2E84935585402A8393F5F50F6F
:1006400015456367B50213F5250019C1BE84B68749
:1006500013F5450001C53A853E87AA8793F2150038
:10066000998989E9639A0200A685BA842E8729A010
:100670009545F9BFE39A02FE3EC893170601C18370
:100680009345F4FF10A33E8593F5F50F1AC616C4E3
:1006900032C23EC00534050542054181135785002D
:1006A0002A974207C24741831246A242218313156B
:1006B000040198A34181135416003243639202044B
:1006C0001373F30F631603022205935585002E95CD
:1006D00093150501C181A181024593C5F5FF93F5ED
:1006E000F50FC93A229542054181218188A089B739
:1006F000330360409375F30F753A42054181F1B7BA
:100700009375F30F453A93150501C18193D7850081
:10071000BE95C205C1B7EFF2BF98B7370A004111C5
:100720009387A7C23EC0F17702C2FD17375400403D
:1007300002C47C839307004002C67C858A8591674A
:10074000130504407C86EF10B05185451305044025
:10075000EF10305F41016FF05F95EFF27F944167DA
:100760007D17511123A2E186375700402AC2AE847B
:1007700032C036C41384418613070740B705020010
:100780003A85EF10B06511C91440B7570040138780
:1007900007401386F6FF10C0F5F218407D55630838
:1007A000071A37550040854513050540EF10F05AEC
:1007B00041677D1718C0370703000507375500400C
:1007C000BA8513050540EF10106011E91440B70712
:1007D0000300138717001386F6FF10C0E5F21840D8
:1007E00079556306071692453755004001461305B3
:1007F0000540EF10305C41677D1718C037070700D0
:100800001307270837550040BA8513050540EF1038
:10081000905B11E91440B707070013872708138678
:10082000F6FF10C0E5F218407555630207123757FE
:100830000040130507408145EF10705537570040C1
:10084000A68513050740EF10305641677D17B704A2
:10085000070018C09384440837550040A685130547
:100860000540EF10505611E518409306F7FF14C0ED
:1008700065F71840715561CFB754004013850440A7
:100880008545EF10D050138504408545EF10F04C9E
:1008900041677D17B704030018C085043755004031
:1008A000A68513050540EF10105211E51840930678
:1008B000F7FF14C065F718406D5551CB9245375579
:1008C0000040054613050540EF10D04E41677D17E7
:1008D000B707030018C09384270037550040A6854A
:1008E00013050540EF10304E11E518409306F7FF51
:1008F00014C065F71C406955B9CBA244A9C03704A0
:1009000000101304040431A0A68513850740EF10DE
:100910001048B757004013850740A285EF10104CD0
:10092000B757004075D1024713850740FD140507EE
:100930003AC0EF10B0478247A38FA7FEC1B7375523
:100940000040130505408545EF10D04201453101B7
:100950006FF0AFF5EFF2CFF441677D17511123A28D
:10096000E186375700402AC4AE8432C036C21384B1
:10097000418613070740B70502003A85EF1010467D
:1009800011C91440B7570040138707401386F6FF7C
:1009900010C0F5F218407D5571CB37570040130554
:1009A00007408545EF10B03E37570040130507401C
:1009B0008545EF10903A41677D1718C0370703004F
:1009C000050737550040BA8513050540EF10B03FC5
:1009D00011E91440B7070300138717001386F6FFC9
:1009E00010C0E5F21840795551C3A2453755004073
:1009F000014613050540EF10F03B41677D1718C015
:100A0000370707001307270837550040BA85130535
:100A10000540EF10503B11E91440B707070013875A
:100A200027081386F6FF10C0E5F2184075551DCF54
:100A300037550040A68513050540EF10F036416795
:100A40007D17B704070018C0938444083755004049
:100A5000A68513050540EF10103711E518409306E1
:100A6000F7FF14C065F71C407155B9EB31016FF009
:100A7000CFE3B7570040B7040010138507409385B4
:100A80000408EF10B035B757004015CD0247138565
:100A90000740370407000C2393041700130444088D
:100AA000EF1090309247FD1793F7F70F3EC237557E
:100AB0000040A28513050540EF10F0306DD926C027
:100AC0009247C5FB01A89385044013850740EF10AA
:100AD000F03011C937550040130505408545EF102A
:100AE0007029014561B78244D9BFEFF26FDB711104
:100AF000D081854613063100B13D11016FF0EFDA68
:100B000093574500638D07109377850F9306800FE9
:100B100001476387D710EFF2AFD8416761117D17A6
:100B2000B75400402AC023A2E186138441869384EF
:100B30000440B70502002685EF10502A11C5184061
:100B40009306F7FF14C075F714407D57D1CE375583
:100B50000040854513050540EF10302041677D17A3
:100B6000B704030018C0850437550040A685130557
:100B70000540EF10502511E518409306F7FF14C00B
:100B800065F714407957ADC28247375500401305C9
:100B9000054093F41700268693F5E70FEF10902198
:100BA0001307001818C0A9E4B704070093842408A9
:100BB000B756004013850640A685EF10D020B756E3
:100BC00000401DC905471C4091E30147B754004050
:100BD0008545138504403AC2EF10D01912470DEF36
:100BE000239A0440938404403A8521016FF0EFCBAF
:100BF000B704030089046DBF18401306F7FF10C047
:100C000071D3B70500109385054013850640EF109A
:100C1000F01C59DD014745BF03070100F1B701474B
:100C20003A858280EFF2CFC74111FD5702C05C8048
:100C30009387C18602C202C4231601002307010064
:100C4000138767032390070023910700239207006F
:100C50009907E399E7FE9387818623900700014671
:100C6000930510071305800623810700EFF06FD965
:100C700081477D563D47B306F10090A28507E39C6E
:100C8000E7FE8A853D4613058006EFF00FDB410144
:100C90006FF0AFC10547A385E1868280EFF24FC0B8
:100CA00083C7B1860111A5C30D661384B18613876E
:100CB000C186814613060682A545B307D6009C234C
:100CC00008108506FD17FD8BAA970A2319072380B4
:100CD000A7FE0355C7FFA380A7FE0355E7FF2381A7
:100CE000A7FEE39CB6FC93878186B8239E23FD462E
:100CF0000A86854513058006FC83230CE100EFF08E
:100D0000CFD52300040005616FF02FBA8967938760
:100D100007723E9508218280EFF28FB89387018594
:100D2000F43303C367009307D00F61112A84814510
:100D300063E4D7009305F00F139516001387018B1A
:100D40003695930727001306F00F05079386018B4E
:100D500006051AC0EFF0DF8C02431307D00F93870C
:100D6000018B1306F00F636467001356230013858D
:100D7000418A1387418A3AC005061387C186814696
:100D80003AC21376F60F9373F40061C0939506018F
:100D90001147C1816368D70A05476388E50A85065C
:100DA00025470505E393E6FE03D7E18A9384E18AAC
:100DB00041E783C6218A03C7318A1385218A938537
:100DC000318AE9E66301041405466301C7143D88CE
:100DD0000546631DC4020D46636AE602130357000D
:100DE000131613001A969382C1860606169683C2BE
:100DF00007002310560083C21700BC23231156009E
:100E00005EA282473E93A9472300F30005071377AC
:100E1000F70F894791E2954763E1E70E98A1142106
:100E20001307800291E251479AA098216315F700B9
:100E3000930700149EA0B93D9E20FD179EA021019E
:100E40006FF0AFA60547E39CE3F4182101C77D17B7
:100E500018A1B1B7924513971600369706072E973B
:100E60008D44814503530700814263786600330354
:100E7000C3409312030193D202018505C2052310DA
:100E80005700C1810907E39F95FC11BF0546E36F39
:100E9000E6F611E7154611C80946054439A039C8D8
:100EA0003D886309C4042546254403C3070083C065
:100EB00017001AC203C3270093171400A2978607CE
:100EC0009382C186420696974182A94393120401F8
:100ED00093D20201E3FCC2F29242239117002392C3
:100EE00067002390570082429907A29223807200E4
:100EF0000504E9BF254615444DBF8506858A238034
:100F0000050014A129BF1146E362E6F0131617008D
:100F10003A961383C18606061A9603C30700231068
:100F2000660003C317002311660003C327002312C2
:100F30006600024629433A9623006600E31904E856
:100F400059BDEFF2EF9593870185AA82A837BC2798
:100F5000511193141500BD8B13971700BA9796077C
:100F60003EC483C70185AA940D4786046384E700C5
:100F70006388020813D45500058889473EC013834F
:100F8000018B139504019307230013071300938625
:100F9000018B1306F00F9305F00F418516C2EFF099
:100FA0002FE8A247930500603385970042054181F1
:100FB000EFF00F9593140501C1809387018B138384
:100FC000018B924221C86387020013F7F2008D461D
:100FD000631FD70090239433AC239387C186138774
:100FE0008701F2AF96B3AEB39907E31CF7FE024751
:100FF000854713441400631CF70031016FF0EF8A3A
:1010000013878186BA97802333348000BDB7854724
:101010003EC0B5B703461300834503008346230053
:1010200093170601C183139505013EC21393060170
:101030004181135303011387C186639F0200938785
:10104000C1861387E70192468AA323926700B6A35D
:101050009907E39AE7FE61BF2EAB52AB76AB41BF77
:10106000EFF20F8403C701850D46130141FDAA86E7
:10107000BE856313C700054783C7518C1386518C07
:1010800032C61386618C32C802C495E31C228507E0
:10109000858B1CA2938701859C330D6613064686BB
:1010A0008607B2979E2332461CA285473EC4B247AC
:1010B0001383C1868C2313F5F600FD1593F7F50F06
:1010C0003ECA5246B24790A33706002083474601E6
:1010D0001306460132C23EC0C2470D66130686851E
:1010E0009C2332D23ECC93171700BA973ED09387F9
:1010F000C1863ECE1384C18681478D647246938437
:10110000C4828142914526D4824363E77700639786
:10111000F316E243638E031E99C66386B700631C11
:10112000B500637AF500825392549693A69383C3D5
:1011300003002310760085028D430906E39672FCB6
:101140007246850793F7F70F190632CE2546E396C8
:10115000C7FA95EA82451386818623840186A30017
:10116000060023010600214693878186637DB60031
:10117000E2451306000F91E131465245A14563F067
:10118000A512BA9790A30246A947631BF60803C6A7
:10119000418C89459387418C814463F6C500930453
:1011A000F6FF93F4F40F84A30E2CC204C1802685AD
:1011B00036CE3ACC1ACAEFE0FFEF42052E2C418121
:1011C00021810AB82685EFE0FFEE420541814E2CD1
:1011D00021812AB82685EFE0FFED42054181F246E4
:1011E00021814AB895EE5243624793076303122C5C
:1011F0001903231DC3FE322C231EC3FE522C231FB2
:10120000C3FEE39667FE138481863A940C202685FC
:1012100036CAEFE03FEA42054181D246218108A06B
:1012200083D7218C1384218C9DEF82471247850739
:1012300093F7F70F1CA399C60D476365F700124794
:1012400091471CA3924725479C236396E706930783
:10125000803E1EA07D572382E18CC2472380070079
:10126000B247238007001E20FD171EA0A24799C386
:10127000EFF05FA21301C1026FE03FE3824463FF1E
:10128000F40499C66386B700E317B5EAE375F5EA97
:10129000A254B383540061BD23100600BDA0524583
:1012A000A145BA97898D3356B640AD45E3CCC5EC20
:1012B00023800700C9BDA944639597009307401F89
:1012C00049BF9305401F31451D2192470AA09C2329
:1012D000E3F2F4F8924723800700ADBFE38D06E404
:1012E0006386B700E319B5E4E377F5E48244E39459
:1012F000F4E4E244E39104E483530600930400021F
:10130000E3FC74F8811323107600854426C425B5C8
:10131000E1FADDB7858963880512EFE27FD8111104
:101320002A84EFF03F97138701855C235833854269
:101330009D8B93962700BE968D6793870783B697FC
:10134000B42381443ECA9D8A36C0931627001307F2
:101350000060158F420741833AC203D6418B124584
:10136000A68516CC32C4EFE0FFD422469305006078
:101370003295EFE03FDB42059387218B1387118B7A
:101380009386018B9305F00F41851306F00FEFF064
:101390002FA99383018B83C70300E2423EC483C716
:1013A00013001387C1863EC683C72300A546138357
:1013B000418B3EC8254581479375F4009143D24047
:1013C00013D61700069693F01700102263930000BF
:1013D00011821D8A631796021DC03306D54013760D
:1013E000F60F11C6814291EDAE8263FCC300224626
:1013F000854212A3324632A3424652A319A0E39873
:1014000002FE850793F7F70F15466393C7009947C8
:10141000FD1693F6F60F1907DDF28247850493F463
:10142000F40FE3FC97F203550300930500600905F0
:1014300042054181EFE0DFCC1383418B2310A300F1
:1014400071016FE09FC682808D89639E0512EFE275
:101450003FC571112A841385818C952C1375F50F66
:1014600019C49377F40009476383E70009819387E0
:10147000018598376376E50A1385818C892C9387DB
:1014800001858C274205418113171500939785012B
:101490003A95E1871D8163D60700B305B04093F507
:1014A000F50F1387018B8605930727009386018B21
:1014B00005071306F00F93F5E50FEFF06F96138510
:1014C000818C312485649387F4FFE98F9305701C28
:1014D0003E853EC0EFE01FC01383018B09CC094756
:1014E000630BE5009376F4008247639BE6029384E6
:1014F000248E63F7F40293171500AA971387C18609
:101500008607BA97034703009AA303471300BAA3B9
:1015100003472300DAA39387818BAA970D4798A3EB
:10152000814415C4894713F7F40F6382F40293765C
:10153000F400638BF600EFF0EFF58504A547E39226
:10154000F4FE11016FE07FB69147E3F6E7FE938763
:10155000818BA697982319C37D1798A38C23939703
:101560001400A69786071387C186BA978D469A23DB
:1015700089C97D17FD169AA393F6F60F8907E5FA38
:101580005DBF0583C5BF8280EFE29FB19387C186AF
:101590001387670323900700239107002392070016
:1015A0009907E399E7FE2381018AA381018A2397A2
:1015B000018A1387418A8147A5463306F700230035
:1015C00006008507E39BD7FE81471387818BA546DD
:1015D0003306F700230006008507E39BD7FEB70715
:1015E00000209305401F3145238A070009222391DB
:1015F000A18C2383018C03C71185A382E18C6FE04A
:10160000DFAA18414C4114450323C5000607B3C7A0
:10161000D50005833D8F1316170093571300398E9D
:10162000B3C76700B18F1397A700318F5CC50CC19A
:1016300054C118C5858B99C71C49BD8E5C4954C1DE
:101640003D8F18C58280EFE2BFA5B717708F9387D3
:10165000E71E1CC95CC1B70779FC9387F7F15CC929
:101660001CC5B70794379387F7DFB796076C7111DE
:101670002A840CC11CCD5CC58544214693865696B0
:10168000639AC400A1442285FD14A53FEDFC11011D
:101690006FE0BFA19387F4FF8D8B8A07A2979C43CD
:1016A00013F734000A0713D5E7012297B6853D8D5D
:1016B0003AC0EFE03FA00247269521461C4385042F
:1016C000A98F1CC3B797076C9386579655BFEFE257
:1016D0003F9D2A843D371C4418404844A183BA9753
:1016E0003D8D858B99C31C4C3D8D6FE01F9CEFE2B7
:1016F0003F9B2A841385818CAE84D13F93150501CD
:10170000C18133858440EFE0FF9A418122954205F3
:1017100041816FE09F9983C7A18E05476381E704EC
:1017200089C789466386D708828001C56302E502BE
:10173000828083C7018585078D8B2388F184A382EE
:10174000018E2383018E130700FC2382E18E8280A9
:10175000138701851C3385079D8B1CB3EDB701C52D
:10176000630AF50282801386018583C5B18E343207
:10177000B397B70013978601B3D6B640E207858AC0
:101780006187E18791C693C7F7FFF98F3CB28280EA
:10179000D98FEDBF1387B18E1C239146850793F730
:1017A000F70F63E4F6001CA3828023000700828009
:1017B00001C56301E504828003C6C18E83C7B18E73
:1017C000138701859386B18E19C686073E975C23E1
:1017D00085075CA382802C33214785079D8B33D6F8
:1017E000F540058A19C29CA282807D171377F70FF6
:1017F0006DF782809387C18E98231337170098A3C3
:101800008280EFE2FF891385818CD1353707002074
:101810000343570183C531851D89814793065701CD
:10182000A1423307F5001D8B33D6E540058A01CA76
:101830006307E30098A2893B05456FE01F87850792
:1018400093F7F70FE39F57FC0145C5BFEFE25F85B4
:101850001385818CAD3D4205418193173500338559
:10186000A74093174500898F9607C1839387071E6A
:1018700037070020231BF7006FE03F8303C7A18ECB
:101880008947631FF70009ED83C7C18E91CB03C75A
:10189000B18E938701850607BA97D8230507D8A389
:1018A0008280370600200347860793771700D1CB45
:1018B00093058607DC2993F61700C1C6B366F700C7
:1018C000898AC1E203C301850D45630CA306EFE2DB
:1018D0002FFD1367870093E78700230CE606138725
:1018E000A18EDCA91C231384A18E850793F7F70F23
:1018F0001CA309476399E70093860185AC3285ED07
:101900002300040019A0E36DF7FEEFF0FFC71820D5
:1019100085476314F700A385018E6FE00FF97D17EB
:101920001377F70F850775D39D8B33D6F540058A5E
:101930007DD69CA2D9BF83C7B18E21479386B18E35
:10194000E5B78280B707002037071900938787071C
:101950001307270DD8C337260000B7260000371716
:1019600000001306268A9386C687130767719305BE
:10197000200D90C7D4C798CB8CCFD0CF94D3D8D3D9
:101980008280EFE2EFF183C7418E01111387418E10
:1019900091CBFD1793F7F70F1CA389E7EFE01FBE6C
:1019A0001387418E83C7E18E9386818E95833EC0D7
:1019B0009E221384E18E9384A18E81CFFD17C207EE
:1019C000C1839EA299E723800400EFE03FBB138709
:1019D000418E1C2090208546850793F7F70F1CA0A9
:1019E000630FD61805C289466301D6229C2005479D
:1019F000638AE738638E072C09476389E73A0561F4
:101A00006FE0AFEA37170140232AD740858BB9CB67
:101A1000EFE01F9D4205418185461387D18E63F615
:101A2000A602931715003E951C2315811375F50F1B
:101A3000939607010905C182636ED50063FFA60076
:101A4000E54663ECF600850721A01C2399C7FD1726
:101A50001CA321A08946E3ECF6FE0C2313058006A7
:101A6000EFE02FF983C73185D1D3B707002003D723
:101A700067019387670105CB3707002003465701AD
:101A8000B7060020938606001317260036971843E2
:101A900019CB914663E9C6000C2001450297B707B0
:101AA00000209387670118200D8B29F39A23454462
:101AB0007D17420741839AA3E36AE4F2EFF08F9D1A
:101AC000B7070020938767019E2363978700153B24
:101AD000E31E05F0A53B19BF21476379F702414793
:101AE0001D8F9307F00FB3D7E74093F7F70F014728
:101AF000C14610083A961CA20507E31CD7FE3D46D6
:101B00000C0813058006EFE04FF3CDB56399E702AB
:101B10009387C186138767032390070023910700EB
:101B2000239207009907E319F7FEB707002003C7C0
:101B300057019307F00FE31BF7EAE13145BD85C379
:101B40001307F00FB357F74093F7F70F0147C1465C
:101B500010083A961CA20507E31CD7FE4DB7814733
:101B60007D5641471408BE9690A28507E39CE7FE88
:101B70003D460C0813058006EFE02FECA1BF93064D
:101B800000FC14A39D8B89EBB717014003A7C74046
:101B90001347170023A6E7409305000413058006AA
:101BA000EFE02FE5EFF00F8F370600209387C18617
:101BB00001471306060093162700B29603A30600FA
:101BC0009386B18E6301030288220C203AC4136508
:101BD00005083EC20293B70700201386070022477C
:101BE00092479386B18E8C229376F70F6399D50036
:101BF0008246858A89C6C14696A3B6A3D6A30507A1
:101C000095469907E319D7FAD5B3930600FC14A3B8
:101C100093F7070289EBB717014003A7C7401347A3
:101C2000170023A6E7409305000413058006EFE0A4
:101C30004FDCEFF02F8683C7C18E138701853AC230
:101C400099CB83C7B18E3EC4EFE08FF9A24712470C
:101C50008607BA97C8B39387C18601473706002025
:101C60009246B432B3D6E640858AA1CE93162700B9
:101C700093050600AE9603A306009386B18E630F0C
:101C8000030088220C203AC6136505083EC402935F
:101C90003247A247370600209386B18E8C22937676
:101CA000F70F639AD5008246858A91C69306000293
:101CB00096A3B6A3D6A3050795469907E312D7FACC
:101CC00035B3239007002391070023920700E5B75F
:101CD000B707002003C757019147E302F7D203C4B7
:101CE0000185938701858C3383C7518E1387518E6D
:101CF0009386818695E71386618E1C2223810600D8
:101D0000A38006008507858B1CA20D66939715009E
:101D100013064686B2979E232384018685831CA3DF
:101D20001C23FD1793F7F70F1CA30947636587046E
:101D300003C5618E1DC50D678605130747862E975F
:101D40001A231305000A7D176384E7001305F00FBB
:101D500011476368F700B307F7403355F540137533
:101D6000F50F36941C20E38CA7C8EFE03FFA08A0DB
:101D7000EFE05FF269B123840186A380060023812E
:101D80000600B5B903C7B18E83C73185B3D7E74025
:101D9000858B1307F00791E301472384E18693873E
:101DA0008186A38007002381070091B903C7C18EF4
:101DB0006DD71307F007D5B7828001A0711122C03B
:101DC0001387018F1E231384018F8507C207C183E8
:101DD0001EA31307F01F6379F700231004009387F5
:101DE000418F9843050798C31E208D8B99E3EFE040
:101DF000FFEAEFE00FE41E20858B99E3EFE0AFD51B
:101E00001E20858B99C3EFE04FD60244B7F700E060
:101E100023A20700110173002030B707002083A719
:101E2000870237F700E0A583FD171CCB23240700AA
:101E3000BD471CC323220700B7E700E0056723A0C6
:101E4000E7108280EFE2CFA54111371401409304DF
:101E500080021307000789474C001305044078826D
:101E60003EC426C6231301000D23130504808947B1
:101E70004C007C82192B9146C1473EC6748236C005
:101E8000130504806D5758C54C000123054778821F
:101E90007956130704403A852326C4404C00F521A7
:101EA000130610084C0037150140708226C6F12930
:101EB0008246B7170140138707404C003A85748269
:101EC000E921194778824C007147371501403AC61D
:101ED0006D29214758C81307000418C8C1471307C4
:101EE00080044C003715014078823EC67929C147ED
:101EF0004C00371501407C8226C641299307000219
:101F00007C824C0093078004371501403EC6B529FA
:101F100041016FE08F99EFE2AF980945CD2DD528AB
:101F2000854537052010EF00C07B05658545130505
:101F300055A3EF0020793937EFE0EFFDB7170140E7
:101F400088471581134515000589EFE02FDDEFE087
:101F50002FB2EFE0CFCBEFE0FFCC1D2183D5E185A1
:101F6000C98D1385818CEFF00FEEEFF0BF9D7535B5
:101F7000EFF08FE137F700E0832707D1DD9B2328BF
:101F8000F7D07300501083D7018F8D8BF5F7EFF0EA
:101F90005F9FCDB7B71702409843B706FFFC1367A2
:101FA000170098C3D843758FD8C39843B706F7FE78
:101FB000FD16758F98C39843B706FCFFFD16758F05
:101FC00098C3D843C176FD16758FD8C337079F00D5
:101FD00098C7984F1367070298CF37170140832699
:101FE00007401306074093F6F6F02320D7408326D8
:101FF000074093E606082320D740094718CA372729
:1020000002401443F19A14C3144314C3D843D8C3F1
:102010008280EFE2EF88371702405C4337040020EC
:102020009146B18B130484026385D700A146638275
:10203000D704B7376E01938707601CC0B7160240FC
:10204000DC420840918313F7F700B707002093871D
:102050008701BA978C23DC4293F5F50F93F70708B5
:102060003357B50081E7EFE0EF862A8718C06FE0AD
:10207000CF835C43B777DC02938707C07DBF01A0A5
:1020800001A001A001A001A001A001A001A001A048
:1020900001A001A001A001A001A001A001A001A038
:1020A00001A001A001A001A001A001A001A001A028
:1020B00001A001A097E1FF1F9381C179138101FB6A
:1020C000170500001305457B97E5FF1F938585F3F2
:1020D00017E6FF1F130606F863FAC5008322050002
:1020E00023A0550011059105E3EAC5FE17E5FF1F82
:1020F000130545F69385C18F6377B500232005004E
:102100001105E36DB5FE93020008739002308D4215
:102110007390428097E2FFFF9382C2EE93E2320017
:1021200073905230EFF01FE7970200009382E2DED7
:102130007390123473002030B72701409387074013
:10214000631EF500EFD2DFF58545130500204D2B0A
:102150008145130500206D236FD03FF582805C41DF
:102160003707F1FF1307F7EF7D8FDC419441A2079A
:10217000D58FD98F5CC11C4537F7F1FF1307D77F87
:10218000D4457D8F9C49D58F94458606D58FD98FB0
:102190001CC55C55370710FF7D177D8FDC29FD17A7
:1021A00093F7F70FD207D98F5CD582801C4589C57C
:1021B00093E717001CC58280F99BEDBF1C4593E790
:1021C00087001CC5828008450D81058982801C45D9
:1021D00093E747001CC582800845098105898280F4
:1021E0001C4591C537075000D98F1CC58280370721
:1021F000B0FF7D17F98FD5BFA54763F8B7041387E4
:1022000065FF931717008322C500BA971D43331348
:10221000F3001343F3FF33735300B397F600B3E7B0
:1022200067005CC5994763E3C7047D1693172600D2
:102230003E965859FD47B397C70093C7F7FFF98FEC
:10224000B395C500DD8D4CD982809397150003238B
:102250000501AE971D473317F7001347F7FF337794
:102260006700B397F6005D8F18C96DBFB14763E291
:10227000C7026516931726003E961859FD47B39777
:10228000C70093C7F7FFF98FB395C500DD8D0CD953
:1022900082804D161317260054553A96FD47B39782
:1022A000C70093C7F7FFF58FB395C500DD8D4CD5FB
:1022B000828068454205418182805C4189C593E7FF
:1022C00007405CC1828093F7F7BFE5BFA54763FB7A
:1022D000B704138765FF931717008322C500BA97C9
:1022E0001D433313F3001343F3FF33735300B397CA
:1022F000F600B3E767005CC5185D09069357470110
:102300008D8B1D8E1376F60F931726003E96FD4794
:10231000B397C70093C7F7FFF98FB395C500DD8D5D
:102320000CDD82809397150003230501AE971D47AE
:102330003317F7001347F7FF33776700B397F600BB
:102340005D8F18C955BF711102C02AC0824793879B
:102350008702BE952EC08247884311014205418104
:10236000828008416D8D3335A00082805C41370743
:1023700000FA7D17F98F5CC15C41DD8D4CC1828014
:10238000B7F7FF1F03A5477C82809C45611122C2DD
:1023900026C013F7070113F3F70001C7D8413363D1
:1023A000E30092211377F60F29C783230500014725
:1023B00013048002930480048546B395E600B37647
:1023C000B6006392D50293122700BD46B39656001D
:1023D00093C6F6FFB3F37600B3125300B3E3720073
:1023E000639787064CC90507A146E317D7FC23204E
:1023F00075001307F00F6378C70483234500A146D7
:1024000013048002930480040547B312D700337786
:1024100056006394E202139726000117BD45B39559
:10242000E50093C5F5FFB3F375003317E300B3631D
:10243000770063928702232A550085064147E3957A
:10244000E6FC232275001244824421018280E39C31
:1024500097F80CC949BFE39297FE23285500F1BFB6
:10246000EFD21FC4111146212A8428002EC06D2AE4
:10247000C246C204C18093F404FCB7450F009385A3
:1024800005243685C20436C2C180EFD0BFC4458D55
:10249000420541814AA01E209246C207C183F99B92
:1024A000C207C1831EA082479043E1679387076AF2
:1024B0009315160063E6C7043685EFD0BFC1AA871F
:1024C0004205418191466373D500914713950701F9
:1024D00041814AAC1E20024793E717001EA01E2030
:1024E00056233227C207C183D18E93F757BFD58FAA
:1024F0001EA016275E27D58F1EA471016FD0FFBACC
:102500008247EA23B167FD176310F502B29536855D
:10251000EFD05FBC420541819317450199E31365F4
:102520001500A1675D8D75B7B387C5008E07B385AC
:10253000C7003685EFD01FBA4205418191675D8D96
:10254000E1BF1E2189C593E717001EA18280C20743
:10255000C183F99BC207C183CDBF1E2189C593E703
:1025600007101EA18280C207C18393F7F7EFC2074D
:10257000C183C5BF1E2189C593E707201EA18280A4
:10258000C207C18393F7F7DFC207C183C5BF1E210E
:1025900089C593E707401EA18280C207C18393F7D4
:1025A000F7BFC207C183C5BF0EA982800A29137570
:1025B000F50F828093F7E50F19C293E71500C20764
:1025C000C1831EA982805E290A2D42055D8D6D8D15
:1025D000220521810D8D133515008280611102C005
:1025E00002C293D7C5012AC23EC08247A205A1817B
:1025F00099CB9247D1073EC29247884321016D8D06
:102600003335A00082809247C181E107EDB723AC4A
:10261000A18E8280B7160240DC4241771307F77F14
:10262000F98F5D8DC8C28280EFD29FA73717024015
:102630005C4391462A84B18B6385D700A146638DA4
:10264000D706B7376E01938707601CC0B7160240E4
:10265000DC42918313F7F700B70700209387070444
:10266000BA978C23DC42184093F5F50F93F70708CF
:102670003355B70081E73A85EFD0DFA548C008C4DD
:1026800048C4B7170240DC43AD83FD8B13D7370036
:102690008A07F18BD98F93F637010D476373D70003
:1026A000D117370700201307C702BA978C23EFD042
:1026B0007FA208C86FD07F9F5C43B777DC02938707
:1026C00007C061B799C5371702401C4F5D8D08CF11
:1026D0008280B7170240984F1345F5FF798D88CF58
:1026E000828099C5371702405C4F5D8D48CF82804C
:1026F000B7170240D84F1345F5FF798DC8CF8280B8
:1027000099C5371702405C475D8D48C78280B7176F
:102710000240D8471345F5FF798DC8C78280000075
:10272000000000000001010101010101010102029C
:10273000020202020202020303030303030303046F
:102740000404040404050505050506060606060737
:10275000070707080808080909090A0A0A0A0B0BEB
:102760000B0C0C0C0D0D0D0E0E0F0F0F1010111188
:102770001112121313141415151616171718181909
:10278000191A1A1B1C1C1D1D1E1F1F20202122226E
:102790002324252526272728292A2B2B2C2D2E2FAD
:1027A0002F30313233343536363738393A3B3C3DC9
:1027B0003E3F4041424344464748494A4B4C4D4FB7
:1027C00050515253555657585A5B5C5E5F60626376
:1027D000646667696A6C6D6E707173747678797B04
:1027E0007C7E8081838486888A8B8D8F919294965B
:1027F000989A9B9D9FA1A3A5A7A9ABADAFB1B3B577
:10280000B7B9BBBDBFC1C4C6C8CACCCFD1D3D6D857
:10281000DADCDFE1E4E6E8EBEDF0F2F5F7FAFCFFF5
:1028200004140111070A1A0D1D0000000000000029
:10283000123455012301234401230123441234009F
:102840000002222243210432104321044321432168
:102850000432102222220000FFF0F000F000FF10EE
:1028600004000000FF00BF007F0055004400290065
:0428700022001D0025
:1028740014130000180D000048140000420F00005B
:1028840060100000FFFF09000102030405060708A9
:10289400010203040506070800366E010204060857
:1028A40004080C10081018201020304020406080CC
:1028B40001020304050607080102030405060708CC
:00000001FF
